BL51 BANKED LINKER/LOCATER V6.22                                                        08/12/2012  15:38:06  PAGE 1


BL51 BANKED LINKER/LOCATER V6.22, INVOKED BY:
C:\KEIL\C51\BIN\BL51.EXE SwanTech_TCPIP_ForSIM900.obj TO SwanTech_TCPIP_ForSIM900 RAMSIZE (256)


MEMORY MODEL: LARGE


INPUT MODULES INCLUDED:
  SwanTech_TCPIP_ForSIM900.obj (SWANTECH_TCPIP_FORSIM900)
  C:\KEIL\C51\LIB\C51L.LIB (?C_STARTUP)
  C:\KEIL\C51\LIB\C51L.LIB (?C?COPY)
  C:\KEIL\C51\LIB\C51L.LIB (?C?CLDOPTR)
  C:\KEIL\C51\LIB\C51L.LIB (?C?CSTOPTR)
  C:\KEIL\C51\LIB\C51L.LIB (?C?IMUL)
  C:\KEIL\C51\LIB\C51L.LIB (?C?ILDIX)
  C:\KEIL\C51\LIB\C51L.LIB (PRINTF)
  C:\KEIL\C51\LIB\C51L.LIB (?C?STRCPY)
  C:\KEIL\C51\LIB\C51L.LIB (STRLEN)
  C:\KEIL\C51\LIB\C51L.LIB (STRSTR)
  C:\KEIL\C51\LIB\C51L.LIB (?C?CLDPTR)
  C:\KEIL\C51\LIB\C51L.LIB (?C?CSTPTR)
  C:\KEIL\C51\LIB\C51L.LIB (?C?IILDX)
  C:\KEIL\C51\LIB\C51L.LIB (?C?PLDIXDATA)
  C:\KEIL\C51\LIB\C51L.LIB (?C?PSTXDATA)
  C:\KEIL\C51\LIB\C51L.LIB (?C?CCASE)
  C:\KEIL\C51\LIB\C51L.LIB (PUTCHAR)


LINK MAP OF MODULE:  SwanTech_TCPIP_ForSIM900 (SWANTECH_TCPIP_FORSIM900)


            TYPE    BASE      LENGTH    RELOCATION   SEGMENT NAME
            -----------------------------------------------------

            * * * * * * *   D A T A   M E M O R Y   * * * * * * *
            REG     0000H     0008H     ABSOLUTE     "REG BANK 0"
            DATA    0008H     0005H     UNIT         _DATA_GROUP_
                    000DH     0013H                  *** GAP ***
            BIT     0020H.0   0001H.1   UNIT         _BIT_GROUP_
                    0021H.1   0000H.7                *** GAP ***
            IDATA   0022H     0001H     UNIT         ?STACK

            * * * * * * *  X D A T A   M E M O R Y  * * * * * * *
            XDATA   0000H     0200H     UNIT         ?XD?SWANTECH_TCPIP_FORSIM900
            XDATA   0200H     0032H     UNIT         _XDATA_GROUP_

            * * * * * * *   C O D E   M E M O R Y   * * * * * * *
            CODE    0000H     0003H     ABSOLUTE     
            CODE    0003H     07D2H     UNIT         ?CO?SWANTECH_TCPIP_FORSIM900
            CODE    07D5H     0365H     UNIT         ?PR?PRINTF?PRINTF
            CODE    0B3AH     02DDH     UNIT         ?C?LIB_CODE
            CODE    0E17H     01AFH     UNIT         ?PR?SWANTECH_TCPIP_CONFIG?SWANTECH_TCPIP_FORSIM900
            CODE    0FC6H     01AAH     UNIT         ?PR?SWANTECH_COMMANDMONITOR?SWANTECH_TCPIP_FORSIM900
            CODE    1170H     011EH     UNIT         ?PR?_UART1_GETSTRING?SWANTECH_TCPIP_FORSIM900
            CODE    128EH     00F7H     UNIT         ?PR?_UART0_GETALINE?SWANTECH_TCPIP_FORSIM900
            CODE    1385H     00BFH     UNIT         ?PR?_STRSTR?STRSTR
            CODE    1444H     00B8H     UNIT         ?PR?_SWANTECH_TCPIP_SEND?SWANTECH_TCPIP_FORSIM900
            CODE    14FCH     00A3H     UNIT         ?PR?_SWANTECH_TCPIP_RECV?SWANTECH_TCPIP_FORSIM900
BL51 BANKED LINKER/LOCATER V6.22                                                      08/12/2012  15:38:06  PAGE 2


            CODE    159FH     0099H     UNIT         ?PR?SWANTECH_TCPIP_CONNECT?SWANTECH_TCPIP_FORSIM900
            CODE    1638H     0054H     UNIT         ?PR?SWANTECH_TCPIP_DISCONNECT?SWANTECH_TCPIP_FORSIM900
            CODE    168CH     0054H     UNIT         ?PR?SWANTECH_TCPIP_NETSHUT?SWANTECH_TCPIP_FORSIM900
            CODE    16E0H     0052H     UNIT         ?PR?_UART1_PUTSTRING?SWANTECH_TCPIP_FORSIM900
            CODE    1732H     0042H     UNIT         ?PR?SWANTECH_COMMANDDISPLAY?SWANTECH_TCPIP_FORSIM900
            CODE    1774H     0041H     UNIT         ?PR?_UART0_PUTSTRING?SWANTECH_TCPIP_FORSIM900
            CODE    17B5H     0039H     UNIT         ?PR?SWANTECH_LOGODISPLAY?SWANTECH_TCPIP_FORSIM900
            CODE    17EEH     0027H     UNIT         ?PR?PUTCHAR?PUTCHAR
            CODE    1815H     001DH     UNIT         ?PR?UART0_INIT?SWANTECH_TCPIP_FORSIM900
            CODE    1832H     0016H     UNIT         ?PR?MAIN?SWANTECH_TCPIP_FORSIM900
            CODE    1848H     0015H     UNIT         ?PR?_STRLEN?STRLEN
            CODE    185DH     0010H     UNIT         ?PR?UART1_INIT?SWANTECH_TCPIP_FORSIM900
            CODE    186DH     000CH     UNIT         ?C_C51STARTUP



OVERLAY MAP OF MODULE:   SwanTech_TCPIP_ForSIM900 (SWANTECH_TCPIP_FORSIM900)


SEGMENT                                             BIT_GROUP          DATA_GROUP          XDATA_GROUP
  +--> CALLED SEGMENT                            START    LENGTH     START    LENGTH     START    LENGTH
--------------------------------------------------------------------------------------------------------
?C_C51STARTUP                                    -----    -----      -----    -----      -----    -----
  +--> ?PR?MAIN?SWANTECH_TCPIP_FORSIM900

?PR?MAIN?SWANTECH_TCPIP_FORSIM900                -----    -----      -----    -----      -----    -----
  +--> ?PR?UART0_INIT?SWANTECH_TCPIP_FORSIM900
  +--> ?PR?UART1_INIT?SWANTECH_TCPIP_FORSIM900
  +--> ?PR?SWANTECH_LOGODISPLAY?SWANTECH_TCP...
  +--> ?PR?SWANTECH_COMMANDDISPLAY?SWANTECH_...
  +--> ?PR?SWANTECH_COMMANDMONITOR?SWANTECH_...

?PR?SWANTECH_LOGODISPLAY?SWANTECH_TCP...         -----    -----      -----    -----      -----    -----
  +--> ?PR?_UART0_PUTSTRING?SWANTECH_TCPIP_F...
  +--> ?CO?SWANTECH_TCPIP_FORSIM900

?PR?_UART0_PUTSTRING?SWANTECH_TCPIP_F...         -----    -----      -----    -----      020AH    0003H
  +--> ?CO?SWANTECH_TCPIP_FORSIM900

?PR?SWANTECH_COMMANDDISPLAY?SWANTECH_...         -----    -----      -----    -----      -----    -----
  +--> ?PR?_UART0_PUTSTRING?SWANTECH_TCPIP_F...
  +--> ?CO?SWANTECH_TCPIP_FORSIM900

?PR?SWANTECH_COMMANDMONITOR?SWANTECH_...         -----    -----      -----    -----      0200H    0005H
  +--> ?CO?SWANTECH_TCPIP_FORSIM900
  +--> ?PR?_UART0_GETALINE?SWANTECH_TCPIP_FO...
  +--> ?PR?_UART0_PUTSTRING?SWANTECH_TCPIP_F...
  +--> ?PR?SWANTECH_TCPIP_CONFIG?SWANTECH_TC...
  +--> ?PR?SWANTECH_TCPIP_CONNECT?SWANTECH_T...
  +--> ?PR?_STRLEN?STRLEN
  +--> ?PR?_SWANTECH_TCPIP_SEND?SWANTECH_TCP...
  +--> ?PR?_SWANTECH_TCPIP_RECV?SWANTECH_TCP...
  +--> ?PR?SWANTECH_TCPIP_DISCONNECT?SWANTEC...
  +--> ?PR?SWANTECH_TCPIP_NETSHUT?SWANTECH_T...
  +--> ?PR?SWANTECH_COMMANDDISPLAY?SWANTECH_...

?PR?_UART0_GETALINE?SWANTECH_TCPIP_FO...         -----    -----      -----    -----      0205H    000CH
BL51 BANKED LINKER/LOCATER V6.22                                                      08/12/2012  15:38:06  PAGE 3



?PR?SWANTECH_TCPIP_CONFIG?SWANTECH_TC...         -----    -----      -----    -----      -----    -----
  +--> ?CO?SWANTECH_TCPIP_FORSIM900
  +--> ?PR?_UART1_PUTSTRING?SWANTECH_TCPIP_F...
  +--> ?PR?_UART1_GETSTRING?SWANTECH_TCPIP_F...
  +--> ?PR?_STRSTR?STRSTR
  +--> ?PR?_UART0_PUTSTRING?SWANTECH_TCPIP_F...

?PR?_UART1_PUTSTRING?SWANTECH_TCPIP_F...         -----    -----      -----    -----      020AH    0003H

?PR?_UART1_GETSTRING?SWANTECH_TCPIP_F...         -----    -----      -----    -----      020AH    000FH

?PR?_STRSTR?STRSTR                               -----    -----      -----    -----      020AH    000CH

?PR?SWANTECH_TCPIP_CONNECT?SWANTECH_T...         -----    -----      -----    -----      -----    -----
  +--> ?CO?SWANTECH_TCPIP_FORSIM900
  +--> ?PR?PRINTF?PRINTF
  +--> ?PR?_UART1_PUTSTRING?SWANTECH_TCPIP_F...
  +--> ?PR?_UART1_GETSTRING?SWANTECH_TCPIP_F...
  +--> ?PR?_STRSTR?STRSTR
  +--> ?PR?_UART0_PUTSTRING?SWANTECH_TCPIP_F...

?PR?PRINTF?PRINTF                                0020H.0  0001H.1    0008H    0005H      020AH    0028H
  +--> ?PR?PUTCHAR?PUTCHAR

?PR?_SWANTECH_TCPIP_SEND?SWANTECH_TCP...         -----    -----      -----    -----      0205H    0005H
  +--> ?CO?SWANTECH_TCPIP_FORSIM900
  +--> ?PR?PRINTF?PRINTF
  +--> ?PR?_UART1_PUTSTRING?SWANTECH_TCPIP_F...
  +--> ?PR?_UART1_GETSTRING?SWANTECH_TCPIP_F...
  +--> ?PR?_STRSTR?STRSTR
  +--> ?PR?_UART0_PUTSTRING?SWANTECH_TCPIP_F...

?PR?_SWANTECH_TCPIP_RECV?SWANTECH_TCP...         -----    -----      -----    -----      0205H    0005H
  +--> ?PR?_UART1_GETSTRING?SWANTECH_TCPIP_F...
  +--> ?CO?SWANTECH_TCPIP_FORSIM900
  +--> ?PR?_STRSTR?STRSTR
  +--> ?PR?_UART1_PUTSTRING?SWANTECH_TCPIP_F...
  +--> ?PR?_UART0_PUTSTRING?SWANTECH_TCPIP_F...

?PR?SWANTECH_TCPIP_DISCONNECT?SWANTEC...         -----    -----      -----    -----      -----    -----
  +--> ?CO?SWANTECH_TCPIP_FORSIM900
  +--> ?PR?PRINTF?PRINTF
  +--> ?PR?_UART1_PUTSTRING?SWANTECH_TCPIP_F...
  +--> ?PR?_UART1_GETSTRING?SWANTECH_TCPIP_F...
  +--> ?PR?_STRSTR?STRSTR
  +--> ?PR?_UART0_PUTSTRING?SWANTECH_TCPIP_F...

?PR?SWANTECH_TCPIP_NETSHUT?SWANTECH_T...         -----    -----      -----    -----      -----    -----
  +--> ?CO?SWANTECH_TCPIP_FORSIM900
  +--> ?PR?PRINTF?PRINTF
  +--> ?PR?_UART1_PUTSTRING?SWANTECH_TCPIP_F...
  +--> ?PR?_UART1_GETSTRING?SWANTECH_TCPIP_F...
  +--> ?PR?_STRSTR?STRSTR
  +--> ?PR?_UART0_PUTSTRING?SWANTECH_TCPIP_F...


BL51 BANKED LINKER/LOCATER V6.22                                                      08/12/2012  15:38:06  PAGE 4



SYMBOL TABLE OF MODULE:  SwanTech_TCPIP_ForSIM900 (SWANTECH_TCPIP_FORSIM900)

  VALUE           TYPE          NAME
  ----------------------------------

  -------         MODULE        SWANTECH_TCPIP_FORSIM900
  C:0000H         SYMBOL        _ICE_DUMMY_
  D:0090H         PUBLIC        P1
  X:0000H         PUBLIC        tcpipBuffer
  D:00A0H         PUBLIC        P2
  D:00B0H         PUBLIC        P3
  D:00A8H         PUBLIC        IE
  D:00B8H         PUBLIC        IP
  B:0098H.0       PUBLIC        RI
  C:128EH         PUBLIC        _Uart0_GetALine
  B:0098H.1       PUBLIC        TI
  C:1732H         PUBLIC        SwanTech_CommandDisplay
  C:1832H         PUBLIC        main
  D:0099H         PUBLIC        SBUF
  D:0087H         PUBLIC        PCON
  C:0FC6H         PUBLIC        SwanTech_CommandMonitor
  C:159FH         PUBLIC        SwanTech_TCPIP_Connect
  D:0098H         PUBLIC        SCON
  D:0089H         PUBLIC        TMOD
  D:0088H         PUBLIC        TCON
  C:0E17H         PUBLIC        SwanTech_TCPIP_Config
  X:0100H         PUBLIC        ttyBuffer
  D:008EH         PUBLIC        AUXR
  C:07D2H         SYMBOL        _?ix1000
  D:00C7H         PUBLIC        IAP_CONTR
  C:1815H         PUBLIC        Uart0_Init
  C:185DH         PUBLIC        Uart1_Init
  B:00A8H.3       PUBLIC        ET1
  C:1184H         PUBLIC        _Uart1_GetString
  D:008DH         PUBLIC        TH1
  D:008BH         PUBLIC        TL1
  C:1638H         PUBLIC        SwanTech_TCPIP_DisConnect
  B:0088H.6       PUBLIC        TR1
  D:009BH         PUBLIC        S2BUF
  C:177AH         PUBLIC        _Uart0_PutString
  C:16E6H         PUBLIC        _Uart1_PutString
  D:009AH         PUBLIC        S2CON
  D:00C8H         PUBLIC        T2CON
  D:009CH         PUBLIC        BRT
  C:144EH         PUBLIC        _SwanTech_TCPIP_Send
  C:17B5H         PUBLIC        SwanTech_LogoDisplay
  C:168CH         PUBLIC        SwanTech_TCPIP_NETShut
  C:14FCH         PUBLIC        _SwanTech_TCPIP_Recv
  D:00D0H         PUBLIC        PSW
  -------         PROC          UART0_INIT
  C:1815H         LINE#         24
  C:1815H         LINE#         25
  C:1815H         LINE#         26
  C:1818H         LINE#         27
  C:181BH         LINE#         28
  C:181EH         LINE#         29
BL51 BANKED LINKER/LOCATER V6.22                                                      08/12/2012  15:38:06  PAGE 5


  C:1821H         LINE#         30
  C:1824H         LINE#         31
  C:1827H         LINE#         32
  C:182AH         LINE#         33
  C:182DH         LINE#         34
  C:182FH         LINE#         35
  C:1831H         LINE#         36
  -------         ENDPROC       UART0_INIT
  C:1774H         SYMBOL        L?0193
  -------         PROC          L?0192
  -------         ENDPROC       L?0192
  C:1774H         SYMBOL        L?0193
  -------         PROC          _UART0_PUTSTRING
  X:020AH         SYMBOL        pString
  -------         DO            
  D:0006H         SYMBOL        i
  -------         ENDDO         
  C:177AH         LINE#         40
  C:1785H         LINE#         41
  C:1785H         LINE#         42
  C:1788H         LINE#         43
  C:179CH         LINE#         44
  C:179CH         LINE#         45
  C:17ADH         LINE#         46
  C:17B0H         LINE#         47
  C:17B2H         LINE#         48
  C:17B4H         LINE#         49
  -------         ENDPROC       _UART0_PUTSTRING
  -------         PROC          _UART0_GETALINE
  X:0205H         SYMBOL        pBuffer
  X:0208H         SYMBOL        nBufferLen
  X:0209H         SYMBOL        nTimeOut
  -------         DO            
  X:020AH         SYMBOL        ch
  X:020BH         SYMBOL        i
  X:020DH         SYMBOL        j
  X:020FH         SYMBOL        k
  -------         ENDDO         
  C:128EH         LINE#         54
  C:129CH         LINE#         55
  C:129CH         LINE#         56
  C:12A1H         LINE#         57
  C:12ADH         LINE#         59
  C:12C3H         LINE#         60
  C:12E4H         LINE#         61
  C:12E4H         LINE#         62
  C:12E4H         LINE#         63
  C:12E4H         LINE#         64
  C:12E7H         LINE#         65
  C:12E7H         LINE#         66
  C:12E9H         LINE#         67
  C:1305H         LINE#         69
  C:130EH         LINE#         70
  C:1311H         LINE#         71
  C:1313H         LINE#         72
  C:1330H         LINE#         73
  C:1330H         LINE#         74
BL51 BANKED LINKER/LOCATER V6.22                                                      08/12/2012  15:38:06  PAGE 6


  C:133EH         LINE#         75
  C:133EH         LINE#         76
  C:133EH         LINE#         77
  C:133EH         LINE#         78
  C:133EH         LINE#         79
  C:1344H         LINE#         80
  C:1346H         LINE#         82
  C:1354H         LINE#         84
  C:136BH         LINE#         85
  C:136BH         LINE#         87
  C:137CH         LINE#         89
  C:1384H         LINE#         90
  -------         ENDPROC       _UART0_GETALINE
  -------         PROC          UART1_INIT
  C:185DH         LINE#         95
  C:185DH         LINE#         96
  C:185DH         LINE#         97
  C:1860H         LINE#         98
  C:1863H         LINE#         99
  C:1866H         LINE#         100
  C:1869H         LINE#         101
  C:186CH         LINE#         102
  -------         ENDPROC       UART1_INIT
  C:16E0H         SYMBOL        L?0191
  -------         PROC          L?0190
  -------         ENDPROC       L?0190
  C:16E0H         SYMBOL        L?0191
  -------         PROC          _UART1_PUTSTRING
  X:020AH         SYMBOL        pString
  -------         DO            
  D:0007H         SYMBOL        i
  -------         ENDDO         
  C:16E6H         LINE#         109
  C:16F1H         LINE#         110
  C:16F1H         LINE#         111
  C:16F3H         LINE#         114
  C:16F3H         LINE#         115
  C:1708H         LINE#         116
  C:1708H         LINE#         118
  C:170AH         LINE#         119
  C:170DH         LINE#         120
  C:170FH         LINE#         122
  C:1727H         LINE#         123
  C:172CH         LINE#         124
  C:172FH         LINE#         125
  C:1731H         LINE#         126
  -------         ENDPROC       _UART1_PUTSTRING
  C:1170H         SYMBOL        L?0187
  C:117EH         SYMBOL        L?0188
  C:117FH         SYMBOL        L?0189
  -------         PROC          L?0186
  -------         ENDPROC       L?0186
  C:1170H         SYMBOL        L?0187
  C:117EH         SYMBOL        L?0188
  C:117FH         SYMBOL        L?0189
  -------         PROC          _UART1_GETSTRING
  X:020AH         SYMBOL        pBuffer
BL51 BANKED LINKER/LOCATER V6.22                                                      08/12/2012  15:38:06  PAGE 7


  X:020DH         SYMBOL        nBufferLen
  X:020FH         SYMBOL        nTimeOut
  -------         DO            
  X:0211H         SYMBOL        i
  X:0213H         SYMBOL        j
  X:0215H         SYMBOL        k
  X:0217H         SYMBOL        nFixedTimeout
  -------         ENDDO         
  C:1184H         LINE#         137
  C:1195H         LINE#         138
  C:1195H         LINE#         139
  C:11A4H         LINE#         143
  C:11ACH         LINE#         145
  C:11D8H         LINE#         146
  C:11D8H         LINE#         147
  C:11F7H         LINE#         148
  C:11F7H         LINE#         149
  C:11FCH         LINE#         150
  C:11FCH         LINE#         151
  C:11FFH         LINE#         152
  C:121EH         LINE#         154
  C:1221H         LINE#         155
  C:1224H         LINE#         156
  C:1226H         LINE#         158
  C:1233H         LINE#         159
  C:123BH         LINE#         160
  C:124EH         LINE#         161
  C:124EH         LINE#         162
  C:124EH         LINE#         163
  C:125EH         LINE#         164
  C:1272H         LINE#         165
  C:128DH         LINE#         167
  C:128DH         LINE#         168
  -------         ENDPROC       _UART1_GETSTRING
  -------         PROC          SWANTECH_LOGODISPLAY
  C:17B5H         LINE#         170
  C:17B5H         LINE#         171
  C:17B5H         LINE#         172
  C:17B8H         LINE#         173
  C:17C1H         LINE#         174
  C:17CAH         LINE#         175
  C:17D3H         LINE#         176
  C:17DCH         LINE#         177
  C:17E5H         LINE#         178
  -------         ENDPROC       SWANTECH_LOGODISPLAY
  -------         PROC          SWANTECH_COMMANDDISPLAY
  C:1732H         LINE#         181
  C:1732H         LINE#         182
  C:1732H         LINE#         183
  C:1735H         LINE#         184
  C:173EH         LINE#         185
  C:1747H         LINE#         186
  C:1750H         LINE#         187
  C:1759H         LINE#         188
  C:1762H         LINE#         189
  C:176BH         LINE#         190
  -------         ENDPROC       SWANTECH_COMMANDDISPLAY
BL51 BANKED LINKER/LOCATER V6.22                                                      08/12/2012  15:38:06  PAGE 8


  -------         PROC          SWANTECH_TCPIP_CONFIG
  C:0E17H         LINE#         198
  C:0E17H         LINE#         199
  C:0E17H         LINE#         202
  C:0E20H         LINE#         203
  C:0E35H         LINE#         204
  C:0E35H         LINE#         205
  C:0E35H         LINE#         206
  C:0E38H         LINE#         207
  C:0E38H         LINE#         208
  C:0E54H         LINE#         209
  C:0E54H         LINE#         210
  C:0E54H         LINE#         211
  C:0E56H         LINE#         212
  C:0E56H         LINE#         215
  C:0E5FH         LINE#         216
  C:0E66H         LINE#         217
  C:0E66H         LINE#         218
  C:0E66H         LINE#         219
  C:0E68H         LINE#         220
  C:0E68H         LINE#         221
  C:0E84H         LINE#         222
  C:0E84H         LINE#         223
  C:0E8AH         LINE#         224
  C:0E8DH         LINE#         225
  C:0E8DH         LINE#         230
  C:0E96H         LINE#         231
  C:0E9DH         LINE#         232
  C:0E9DH         LINE#         233
  C:0EA3H         LINE#         234
  C:0EA6H         LINE#         235
  C:0EA6H         LINE#         236
  C:0EC2H         LINE#         237
  C:0EC2H         LINE#         238
  C:0EC8H         LINE#         239
  C:0ECBH         LINE#         240
  C:0ECBH         LINE#         243
  C:0ED4H         LINE#         244
  C:0EDBH         LINE#         245
  C:0EDBH         LINE#         246
  C:0EE1H         LINE#         247
  C:0EE4H         LINE#         248
  C:0EE4H         LINE#         249
  C:0F00H         LINE#         250
  C:0F00H         LINE#         251
  C:0F06H         LINE#         252
  C:0F09H         LINE#         253
  C:0F09H         LINE#         256
  C:0F12H         LINE#         257
  C:0F19H         LINE#         258
  C:0F19H         LINE#         259
  C:0F1FH         LINE#         260
  C:0F22H         LINE#         261
  C:0F22H         LINE#         262
  C:0F3EH         LINE#         263
  C:0F3EH         LINE#         264
  C:0F44H         LINE#         265
BL51 BANKED LINKER/LOCATER V6.22                                                      08/12/2012  15:38:06  PAGE 9


  C:0F47H         LINE#         266
  C:0F47H         LINE#         269
  C:0F50H         LINE#         270
  C:0F57H         LINE#         271
  C:0F57H         LINE#         272
  C:0F5DH         LINE#         273
  C:0F5FH         LINE#         274
  C:0F5FH         LINE#         275
  C:0F7BH         LINE#         276
  C:0F7BH         LINE#         277
  C:0F81H         LINE#         278
  C:0F83H         LINE#         279
  C:0F83H         LINE#         282
  C:0F8CH         LINE#         283
  C:0F93H         LINE#         284
  C:0F93H         LINE#         285
  C:0F99H         LINE#         286
  C:0F9BH         LINE#         287
  C:0F9BH         LINE#         288
  C:0FB7H         LINE#         289
  C:0FB7H         LINE#         290
  C:0FC0H         LINE#         291
  C:0FC3H         LINE#         292
  C:0FC3H         LINE#         294
  C:0FC5H         LINE#         295
  -------         ENDPROC       SWANTECH_TCPIP_CONFIG
  -------         PROC          SWANTECH_TCPIP_CONNECT
  C:159FH         LINE#         302
  C:159FH         LINE#         303
  C:159FH         LINE#         305
  C:15CEH         LINE#         306
  C:15D1H         LINE#         307
  C:15D8H         LINE#         308
  C:15D8H         LINE#         309
  C:15D8H         LINE#         310
  C:15DAH         LINE#         311
  C:15DAH         LINE#         312
  C:15F6H         LINE#         313
  C:15F6H         LINE#         314
  C:15FCH         LINE#         315
  C:15FEH         LINE#         316
  C:15FEH         LINE#         319
  C:1605H         LINE#         320
  C:1605H         LINE#         321
  C:160BH         LINE#         322
  C:160DH         LINE#         323
  C:160DH         LINE#         324
  C:1629H         LINE#         325
  C:1629H         LINE#         326
  C:1632H         LINE#         327
  C:1635H         LINE#         328
  C:1635H         LINE#         330
  C:1637H         LINE#         331
  -------         ENDPROC       SWANTECH_TCPIP_CONNECT
  -------         PROC          SWANTECH_TCPIP_DISCONNECT
  C:1638H         LINE#         338
  C:1638H         LINE#         339
BL51 BANKED LINKER/LOCATER V6.22                                                      08/12/2012  15:38:06  PAGE 10


  C:1638H         LINE#         341
  C:164FH         LINE#         342
  C:1652H         LINE#         343
  C:1659H         LINE#         344
  C:1659H         LINE#         345
  C:165FH         LINE#         346
  C:1661H         LINE#         347
  C:1661H         LINE#         348
  C:167DH         LINE#         349
  C:167DH         LINE#         350
  C:1686H         LINE#         351
  C:1689H         LINE#         352
  C:1689H         LINE#         354
  C:168BH         LINE#         355
  -------         ENDPROC       SWANTECH_TCPIP_DISCONNECT
  -------         PROC          SWANTECH_TCPIP_NETSHUT
  C:168CH         LINE#         362
  C:168CH         LINE#         363
  C:168CH         LINE#         365
  C:16A3H         LINE#         366
  C:16A6H         LINE#         367
  C:16ADH         LINE#         368
  C:16ADH         LINE#         369
  C:16B3H         LINE#         370
  C:16B5H         LINE#         371
  C:16B5H         LINE#         372
  C:16D1H         LINE#         373
  C:16D1H         LINE#         374
  C:16DAH         LINE#         375
  C:16DDH         LINE#         376
  C:16DDH         LINE#         378
  C:16DFH         LINE#         379
  -------         ENDPROC       SWANTECH_TCPIP_NETSHUT
  -------         PROC          L?0194
  -------         ENDPROC       L?0194
  -------         PROC          _SWANTECH_TCPIP_SEND
  X:0205H         SYMBOL        pBuffer
  X:0208H         SYMBOL        nBufferLen
  C:144EH         LINE#         387
  C:145FH         LINE#         388
  C:145FH         LINE#         391
  C:147CH         LINE#         392
  C:147FH         LINE#         393
  C:1486H         LINE#         394
  C:1486H         LINE#         395
  C:1486H         LINE#         396
  C:1488H         LINE#         397
  C:1488H         LINE#         398
  C:14A4H         LINE#         399
  C:14A4H         LINE#         400
  C:14AAH         LINE#         401
  C:14ACH         LINE#         402
  C:14ACH         LINE#         405
  C:14BAH         LINE#         406
  C:14C1H         LINE#         407
  C:14C1H         LINE#         408
  C:14C7H         LINE#         409
BL51 BANKED LINKER/LOCATER V6.22                                                      08/12/2012  15:38:06  PAGE 11


  C:14C9H         LINE#         410
  C:14C9H         LINE#         411
  C:14E5H         LINE#         412
  C:14E5H         LINE#         413
  C:14EEH         LINE#         414
  C:14F3H         LINE#         415
  C:14F3H         LINE#         417
  C:14FBH         LINE#         418
  -------         ENDPROC       _SWANTECH_TCPIP_SEND
  -------         PROC          _SWANTECH_TCPIP_RECV
  X:0205H         SYMBOL        pBuffer
  X:0208H         SYMBOL        nBufferLen
  C:14FCH         LINE#         426
  C:150DH         LINE#         427
  C:150DH         LINE#         429
  C:1523H         LINE#         430
  C:1523H         LINE#         431
  C:1523H         LINE#         432
  C:1525H         LINE#         433
  C:1525H         LINE#         434
  C:1541H         LINE#         435
  C:1541H         LINE#         436
  C:1547H         LINE#         437
  C:1549H         LINE#         438
  C:1549H         LINE#         441
  C:1552H         LINE#         442
  C:1568H         LINE#         443
  C:1568H         LINE#         444
  C:156EH         LINE#         445
  C:1570H         LINE#         446
  C:1570H         LINE#         447
  C:158CH         LINE#         448
  C:158CH         LINE#         449
  C:1595H         LINE#         450
  C:159AH         LINE#         451
  C:159AH         LINE#         453
  C:159EH         LINE#         454
  -------         ENDPROC       _SWANTECH_TCPIP_RECV
  -------         PROC          SWANTECH_COMMANDMONITOR
  -------         DO            
  X:0200H         SYMBOL        bFinishConfig
  X:0201H         SYMBOL        bFinishConnect
  X:0202H         SYMBOL        buffer
  -------         ENDDO         
  C:0FC6H         LINE#         456
  C:0FC6H         LINE#         457
  C:0FC6H         LINE#         458
  C:0FCBH         LINE#         459
  C:0FCDH         LINE#         460
  C:0FDFH         LINE#         462
  C:0FDFH         LINE#         463
  C:0FDFH         LINE#         464
  C:0FEFH         LINE#         467
  C:0FFBH         LINE#         468
  C:0FFEH         LINE#         470
  C:1001H         LINE#         471
  C:1008H         LINE#         472
BL51 BANKED LINKER/LOCATER V6.22                                                      08/12/2012  15:38:06  PAGE 12


  C:1008H         LINE#         473
  C:100EH         LINE#         474
  C:100EH         LINE#         475
  C:1013H         LINE#         476
  C:1019H         LINE#         477
  C:101CH         LINE#         479
  C:101CH         LINE#         480
  C:1022H         LINE#         481
  C:1028H         LINE#         482
  C:1028H         LINE#         483
  C:102BH         LINE#         484
  C:1033H         LINE#         485
  C:1033H         LINE#         486
  C:1039H         LINE#         487
  C:1042H         LINE#         488
  C:1048H         LINE#         489
  C:1048H         LINE#         490
  C:104DH         LINE#         491
  C:1053H         LINE#         492
  C:1056H         LINE#         494
  C:1056H         LINE#         495
  C:105CH         LINE#         496
  C:1062H         LINE#         497
  C:1062H         LINE#         498
  C:1065H         LINE#         499
  C:106DH         LINE#         500
  C:106DH         LINE#         501
  C:107CH         LINE#         502
  C:1082H         LINE#         503
  C:108BH         LINE#         504
  C:109DH         LINE#         505
  C:10A6H         LINE#         507
  C:10ACH         LINE#         508
  C:10AFH         LINE#         509
  C:10B7H         LINE#         510
  C:10B7H         LINE#         511
  C:10C6H         LINE#         512
  C:10CCH         LINE#         513
  C:10D5H         LINE#         515
  C:10D5H         LINE#         516
  C:10E7H         LINE#         517
  C:10EFH         LINE#         519
  C:10F8H         LINE#         521
  C:1101H         LINE#         523
  C:1114H         LINE#         524
  C:111CH         LINE#         526
  C:1122H         LINE#         527
  C:1122H         LINE#         528
  C:1124H         LINE#         529
  C:112CH         LINE#         530
  C:112CH         LINE#         531
  C:1132H         LINE#         532
  C:113AH         LINE#         533
  C:1142H         LINE#         534
  C:1148H         LINE#         536
  C:114CH         LINE#         537
  C:114EH         LINE#         538
BL51 BANKED LINKER/LOCATER V6.22                                                      08/12/2012  15:38:06  PAGE 13


  C:1155H         LINE#         539
  C:1155H         LINE#         540
  C:115DH         LINE#         541
  C:1163H         LINE#         543
  C:116AH         LINE#         544
  C:116AH         LINE#         546
  C:116DH         LINE#         547
  -------         ENDPROC       SWANTECH_COMMANDMONITOR
  -------         PROC          MAIN
  C:1832H         LINE#         550
  C:1832H         LINE#         551
  C:1832H         LINE#         552
  C:1835H         LINE#         553
  C:1838H         LINE#         555
  C:1838H         LINE#         556
  C:1838H         LINE#         557
  C:183BH         LINE#         558
  C:183BH         LINE#         559
  C:183DH         LINE#         560
  C:1840H         LINE#         561
  C:1843H         LINE#         562
  C:1843H         LINE#         563
  C:1843H         LINE#         564
  C:1843H         LINE#         566
  -------         ENDPROC       MAIN
  -------         ENDMOD        SWANTECH_TCPIP_FORSIM900

  -------         MODULE        ?C?COPY
  C:0C0AH         PUBLIC        ?C?COPY
  -------         ENDMOD        ?C?COPY

  -------         MODULE        ?C?CLDOPTR
  C:0C30H         PUBLIC        ?C?CLDOPTR
  -------         ENDMOD        ?C?CLDOPTR

  -------         MODULE        ?C?CSTOPTR
  C:0C5DH         PUBLIC        ?C?CSTOPTR
  -------         ENDMOD        ?C?CSTOPTR

  -------         MODULE        ?C?IMUL
  C:0C7FH         PUBLIC        ?C?IMUL
  -------         ENDMOD        ?C?IMUL

  -------         MODULE        ?C?ILDIX
  C:0C91H         PUBLIC        ?C?ILDIX
  -------         ENDMOD        ?C?ILDIX

  -------         MODULE        PRINTF
  X:020AH         PUBLIC        ?_PRINTF517?BYTE
  X:020AH         PUBLIC        ?_PRINTF?BYTE
  X:020AH         PUBLIC        ?_SPRINTF517?BYTE
  X:020AH         PUBLIC        ?_SPRINTF?BYTE
  C:0840H         PUBLIC        _PRINTF
  C:0840H         PUBLIC        _PRINTF517
  C:083AH         PUBLIC        _SPRINTF
  C:083AH         PUBLIC        _SPRINTF517
  -------         ENDMOD        PRINTF
BL51 BANKED LINKER/LOCATER V6.22                                                      08/12/2012  15:38:06  PAGE 14



  -------         MODULE        ?C?STRCPY
  C:0D73H         PUBLIC        ?C?STRCPY
  -------         ENDMOD        ?C?STRCPY

  -------         MODULE        STRLEN
  C:1848H         PUBLIC        _STRLEN
  -------         ENDMOD        STRLEN

  -------         MODULE        STRSTR
  X:020AH         PUBLIC        ?_strstr?BYTE
  C:1385H         PUBLIC        _strstr
  -------         ENDMOD        STRSTR

  -------         MODULE        ?C?CLDPTR
  C:0D90H         PUBLIC        ?C?CLDPTR
  -------         ENDMOD        ?C?CLDPTR

  -------         MODULE        ?C?CSTPTR
  C:0DA9H         PUBLIC        ?C?CSTPTR
  -------         ENDMOD        ?C?CSTPTR

  -------         MODULE        ?C?IILDX
  C:0DBBH         PUBLIC        ?C?IILDX
  -------         ENDMOD        ?C?IILDX

  -------         MODULE        ?C?PLDIXDATA
  C:0DD1H         PUBLIC        ?C?PLDIXDATA
  -------         ENDMOD        ?C?PLDIXDATA

  -------         MODULE        ?C?PSTXDATA
  C:0DE8H         PUBLIC        ?C?PSTXDATA
  -------         ENDMOD        ?C?PSTXDATA

  -------         MODULE        ?C?CCASE
  C:0DF1H         PUBLIC        ?C?CCASE
  -------         ENDMOD        ?C?CCASE

  -------         MODULE        PUTCHAR
  C:17EEH         PUBLIC        _PUTCHAR
  -------         ENDMOD        PUTCHAR

Program Size: data=15.1 xdata=562 code=6265
LINK/LOCATE RUN COMPLETE.  0 WARNING(S),  0 ERROR(S)
